Archive member included because of file (symbol)

/usr/lib/gcc/avr/4.3.2/avr25/libgcc.a(_exit.o)
                              /usr/lib/gcc/avr/4.3.2/../../../avr/lib/avr25/crttn2313.o (exit)
/usr/lib/gcc/avr/4.3.2/avr25/libgcc.a(_copy_data.o)
                              ./lcd4.o (__do_copy_data)
/usr/lib/gcc/avr/4.3.2/avr25/libgcc.a(_clear_bss.o)
                              ./lcd4.o (__do_clear_bss)

Memory Configuration

Name             Origin             Length             Attributes
text             0x00000000         0x00002000         xr
data             0x00800060         0x0000ffa0         rw !x
eeprom           0x00810000         0x00010000         rw !x
fuse             0x00820000         0x00000400         rw !x
lock             0x00830000         0x00000400         rw !x
signature        0x00840000         0x00000400         rw !x
*default*        0x00000000         0xffffffff

Linker script and memory map

LOAD /usr/lib/gcc/avr/4.3.2/../../../avr/lib/avr25/crttn2313.o
LOAD ./lcd4.o
LOAD ./lcd_wait.o
LOAD ./lcdtest.o
LOAD /usr/lib/gcc/avr/4.3.2/avr25/libgcc.a
LOAD /usr/lib/gcc/avr/4.3.2/../../../avr/lib/avr25/libc.a
LOAD /usr/lib/gcc/avr/4.3.2/avr25/libgcc.a

.hash
 *(.hash)

.dynsym
 *(.dynsym)

.dynstr
 *(.dynstr)

.gnu.version
 *(.gnu.version)

.gnu.version_d
 *(.gnu.version_d)

.gnu.version_r
 *(.gnu.version_r)

.rel.init
 *(.rel.init)

.rela.init
 *(.rela.init)

.rel.text
 *(.rel.text)
 *(.rel.text.*)
 *(.rel.gnu.linkonce.t*)

.rela.text
 *(.rela.text)
 *(.rela.text.*)
 *(.rela.gnu.linkonce.t*)

.rel.fini
 *(.rel.fini)

.rela.fini
 *(.rela.fini)

.rel.rodata
 *(.rel.rodata)
 *(.rel.rodata.*)
 *(.rel.gnu.linkonce.r*)

.rela.rodata
 *(.rela.rodata)
 *(.rela.rodata.*)
 *(.rela.gnu.linkonce.r*)

.rel.data
 *(.rel.data)
 *(.rel.data.*)
 *(.rel.gnu.linkonce.d*)

.rela.data
 *(.rela.data)
 *(.rela.data.*)
 *(.rela.gnu.linkonce.d*)

.rel.ctors
 *(.rel.ctors)

.rela.ctors
 *(.rela.ctors)

.rel.dtors
 *(.rel.dtors)

.rela.dtors
 *(.rela.dtors)

.rel.got
 *(.rel.got)

.rela.got
 *(.rela.got)

.rel.bss
 *(.rel.bss)

.rela.bss
 *(.rela.bss)

.rel.plt
 *(.rel.plt)

.rela.plt
 *(.rela.plt)

.text           0x00000000      0x3f2
 *(.vectors)
 .vectors       0x00000000       0x26 /usr/lib/gcc/avr/4.3.2/../../../avr/lib/avr25/crttn2313.o
                0x00000000                __vectors
                0x00000000                __vector_default
 *(.vectors)
 *(.progmem.gcc*)
 *(.progmem*)
                0x00000026                . = ALIGN (0x2)
                0x00000026                __trampolines_start = .
 *(.trampolines)
 .trampolines   0x00000026        0x0 linker stubs
 *(.trampolines*)
                0x00000026                __trampolines_end = .
 *(.jumptables)
 *(.jumptables*)
 *(.lowtext)
 *(.lowtext*)
                0x00000026                __ctors_start = .
 *(.ctors)
                0x00000026                __ctors_end = .
                0x00000026                __dtors_start = .
 *(.dtors)
                0x00000026                __dtors_end = .
 SORT(*)(.ctors)
 SORT(*)(.dtors)
 *(.init0)
 .init0         0x00000026        0x0 /usr/lib/gcc/avr/4.3.2/../../../avr/lib/avr25/crttn2313.o
                0x00000026                __init
 *(.init0)
 *(.init1)
 *(.init1)
 *(.init2)
 .init2         0x00000026        0x8 /usr/lib/gcc/avr/4.3.2/../../../avr/lib/avr25/crttn2313.o
 *(.init2)
 *(.init3)
 *(.init3)
 *(.init4)
 .init4         0x0000002e       0x16 /usr/lib/gcc/avr/4.3.2/avr25/libgcc.a(_copy_data.o)
                0x0000002e                __do_copy_data
 .init4         0x00000044       0x10 /usr/lib/gcc/avr/4.3.2/avr25/libgcc.a(_clear_bss.o)
                0x00000044                __do_clear_bss
 *(.init4)
 *(.init5)
 *(.init5)
 *(.init6)
 *(.init6)
 *(.init7)
 *(.init7)
 *(.init8)
 *(.init8)
 *(.init9)
 .init9         0x00000054        0x4 /usr/lib/gcc/avr/4.3.2/../../../avr/lib/avr25/crttn2313.o
 *(.init9)
 *(.text)
 .text          0x00000058        0x2 /usr/lib/gcc/avr/4.3.2/../../../avr/lib/avr25/crttn2313.o
                0x00000058                __vector_1
                0x00000058                __vector_12
                0x00000058                __bad_interrupt
                0x00000058                __vector_6
                0x00000058                __vector_3
                0x00000058                __vector_11
                0x00000058                __vector_13
                0x00000058                __vector_17
                0x00000058                __vector_7
                0x00000058                __vector_5
                0x00000058                __vector_4
                0x00000058                __vector_9
                0x00000058                __vector_2
                0x00000058                __vector_15
                0x00000058                __vector_8
                0x00000058                __vector_14
                0x00000058                __vector_10
                0x00000058                __vector_16
                0x00000058                __vector_18
 .text          0x0000005a      0x2e6 ./lcd4.o
                0x0000014e                lcd_write
                0x0000010c                lcd_1s
                0x000002c2                lcd_blank_line
                0x000000e6                lcd_5ms
                0x00000132                lcd_instruct
                0x0000005a                lcd_init
 .text          0x00000340       0x46 ./lcd_wait.o
                0x00000340                wait_100us
 .text          0x00000386       0x68 ./lcdtest.o
                0x00000386                main
 .text          0x000003ee        0x0 /usr/lib/gcc/avr/4.3.2/avr25/libgcc.a(_exit.o)
 .text          0x000003ee        0x0 /usr/lib/gcc/avr/4.3.2/avr25/libgcc.a(_copy_data.o)
 .text          0x000003ee        0x0 /usr/lib/gcc/avr/4.3.2/avr25/libgcc.a(_clear_bss.o)
                0x000003ee                . = ALIGN (0x2)
 *(.text.*)
 .text.libgcc   0x000003ee        0x0 /usr/lib/gcc/avr/4.3.2/avr25/libgcc.a(_exit.o)
 .text.libgcc   0x000003ee        0x0 /usr/lib/gcc/avr/4.3.2/avr25/libgcc.a(_copy_data.o)
 .text.libgcc   0x000003ee        0x0 /usr/lib/gcc/avr/4.3.2/avr25/libgcc.a(_clear_bss.o)
                0x000003ee                . = ALIGN (0x2)
 *(.fini9)
 .fini9         0x000003ee        0x0 /usr/lib/gcc/avr/4.3.2/avr25/libgcc.a(_exit.o)
                0x000003ee                exit
                0x000003ee                _exit
 *(.fini9)
 *(.fini8)
 *(.fini8)
 *(.fini7)
 *(.fini7)
 *(.fini6)
 *(.fini6)
 *(.fini5)
 *(.fini5)
 *(.fini4)
 *(.fini4)
 *(.fini3)
 *(.fini3)
 *(.fini2)
 *(.fini2)
 *(.fini1)
 *(.fini1)
 *(.fini0)
 .fini0         0x000003ee        0x4 /usr/lib/gcc/avr/4.3.2/avr25/libgcc.a(_exit.o)
 *(.fini0)
                0x000003f2                _etext = .

.data           0x00800060        0x0 load address 0x000003f2
                0x00800060                PROVIDE (__data_start, .)
 *(.data)
 .data          0x00800060        0x0 /usr/lib/gcc/avr/4.3.2/../../../avr/lib/avr25/crttn2313.o
 .data          0x00800060        0x0 ./lcd4.o
 .data          0x00800060        0x0 ./lcd_wait.o
 .data          0x00800060        0x0 ./lcdtest.o
 .data          0x00800060        0x0 /usr/lib/gcc/avr/4.3.2/avr25/libgcc.a(_exit.o)
 .data          0x00800060        0x0 /usr/lib/gcc/avr/4.3.2/avr25/libgcc.a(_copy_data.o)
 .data          0x00800060        0x0 /usr/lib/gcc/avr/4.3.2/avr25/libgcc.a(_clear_bss.o)
 *(.data*)
 *(.rodata)
 *(.rodata*)
 *(.gnu.linkonce.d*)
                0x00800060                . = ALIGN (0x2)
                0x00800060                _edata = .
                0x00800060                PROVIDE (__data_end, .)

.bss            0x00800060        0x0 load address 0x000003f2
                0x00800060                PROVIDE (__bss_start, .)
 *(.bss)
 .bss           0x00800060        0x0 /usr/lib/gcc/avr/4.3.2/../../../avr/lib/avr25/crttn2313.o
 .bss           0x00800060        0x0 ./lcd4.o
 .bss           0x00800060        0x0 ./lcd_wait.o
 .bss           0x00800060        0x0 ./lcdtest.o
 .bss           0x00800060        0x0 /usr/lib/gcc/avr/4.3.2/avr25/libgcc.a(_exit.o)
 .bss           0x00800060        0x0 /usr/lib/gcc/avr/4.3.2/avr25/libgcc.a(_copy_data.o)
 .bss           0x00800060        0x0 /usr/lib/gcc/avr/4.3.2/avr25/libgcc.a(_clear_bss.o)
 *(.bss*)
 *(COMMON)
                0x00800060                PROVIDE (__bss_end, .)
                0x000003f2                __data_load_start = LOADADDR (.data)
                0x000003f2                __data_load_end = (__data_load_start + SIZEOF (.data))

.noinit         0x00800060        0x0
                0x00800060                PROVIDE (__noinit_start, .)
 *(.noinit*)
                0x00800060                PROVIDE (__noinit_end, .)
                0x00800060                _end = .
                0x00800060                PROVIDE (__heap_start, .)

.eeprom         0x00810000        0x0
 *(.eeprom*)
                0x00810000                __eeprom_end = .

.fuse
 *(.fuse)
 *(.lfuse)
 *(.hfuse)
 *(.efuse)

.lock
 *(.lock*)

.signature
 *(.signature*)

.stab           0x00000000     0x1158
 *(.stab)
 .stab          0x00000000      0x69c /usr/lib/gcc/avr/4.3.2/../../../avr/lib/avr25/crttn2313.o
 .stab          0x0000069c      0x6fc ./lcd4.o
                                0x708 (size before relaxing)
 .stab          0x00000d98      0x180 ./lcd_wait.o
                                0x348 (size before relaxing)
 .stab          0x00000f18      0x240 ./lcdtest.o
                                0x408 (size before relaxing)

.stabstr        0x00000000      0x7ee
 *(.stabstr)
 .stabstr       0x00000000      0x7ee /usr/lib/gcc/avr/4.3.2/../../../avr/lib/avr25/crttn2313.o

.stab.excl
 *(.stab.excl)

.stab.exclstr
 *(.stab.exclstr)

.stab.index
 *(.stab.index)

.stab.indexstr
 *(.stab.indexstr)

.comment
 *(.comment)

.debug
 *(.debug)

.line
 *(.line)

.debug_srcinfo
 *(.debug_srcinfo)

.debug_sfnames
 *(.debug_sfnames)

.debug_aranges
 *(.debug_aranges)

.debug_pubnames
 *(.debug_pubnames)

.debug_info
 *(.debug_info)
 *(.gnu.linkonce.wi.*)

.debug_abbrev
 *(.debug_abbrev)

.debug_line
 *(.debug_line)

.debug_frame
 *(.debug_frame)

.debug_str
 *(.debug_str)

.debug_loc
 *(.debug_loc)

.debug_macinfo
 *(.debug_macinfo)
OUTPUT(LCD4.elf elf32-avr)
LOAD linker stubs
